:020000040000FA
:100000008316FF2390008630810083120130850023
:100010000130A1000C3083168500831214282108BA
:1000200085008101851D5728811A0F28051914287C
:1000300000000000000000000000000000000000C0
:100040000830A300A0010630A4000000A40B25285E
:100050000310A00C0519A017A30B23280630A40039
:10006000A40B3028051D14282008F83A031952283B
:100070002008FA3A031948282008FB3A03194C28AB
:100080002008FC3A031D1428A11221088500142819
:10009000A116210885001428A11621080238850020
:1000A00081011428210810388500810114283E3070
:1000B0008316850083120301A20085190828051EF6
:1000C0007428221C7828851E6828A21C6F285D28A9
:1000D000A21C5D2822080139A200FC307C282208DD
:1000E0000238A200FA307C2822080239A2006328D4
:1000F00022080138A200F830A30085010830A500CD
:10010000A50B80280830A4000000230885000730D4
:10011000A500A50B89280314A30C00000000A40B64
:06012000852800005D28A7
:02400E00D43F9D
:00000001FF
